:0A00000075817F7401F58F02000E78
:10000B0002023FC229C2287400900010F090001128
:10001B00F0900012F0900013F0900014F074009028
:10002B000016F07401900017F07402900018F07431
:10003B0003900019F0740490001AF0740590001BE3
:10004B00F0740690001CF0740790001DF07408907B
:10005B00001EF0740990001FF0740A900020F074D9
:10006B000B900021F07400900031F0900032F09072
:10007B000033F0900034F0900035F0740290002FB4
:10008B00F07402900030F090003779FF7400F0A309
:10009B00D9FA90013679FF7400F0A3D9FA900237A0
:1000AB0079FF7400F0A3D9FA90033679CD7400F080
:1000BB00A3D9FA120EBE7563FF7564FF7565FF75E4
:1000CB00460075470075700075670075710075689F
:1000DB0000C208C2097540007541007542007543A6
:1000EB0000754C00754D00756F027548FF75490A18
:1000FB0085483C85493D754A7F754B01854A44854A
:10010B004B45755500D226C2C175A012C2B1C2B300
:10011B00C2B4C2B5C2B6C281C2B2C2841206A512A3
:10012B0006C41206E312070212081975597F755A95
:10013B007F755B7F755D00755E00755F001201EF6B
:10014B001205A01205FB12216F75720075730175F4
:10015B0071001216BD121F0D121F18D20FD22CC216
:10016B002E12236E12081912240012252C121F0DA9
:10017B00121F181208BC120B0D120EDB12153012C7
:10018B001548121CC8121CAD1223A302016C85600A
:10019B0090C2A7C2C0D2C022856190D2A7C2C0D2E2
:1001AB00C022C285C281C2B2C284E56379081392B0
:1001BB0083C285D285D9F7D2810000C281E56479EB
:1001CB0008139283C285D285D9F7D2B20000C2B28E
:1001DB00E5657908139283C285D285D9F7D284005D
:1001EB0000C28422758790758922758DFC758BFCF6
:1001FB00759850C299C298758C38758A38753906BE
:10020B00753A04753B0590FF9C8582CA8583CB8527
:10021B0082CC8583CDC200C201D28CD2A9D2AF22AF
:10022B00783279320000D9FCD8F822780A790FD9C4
:10023B00FED8FA22C2AFC0E0C0D0E5F0C0E0E58244
:10024B00C0E0E583C0E0E574C0E0E8C0E0E9C0E0F1
:10025B00EAC0E0EBC0E01206E31224D81224EC1241
:10026B0011B8D544107544FFD5450A854A44854BD2
:10027B0045D223D22712241A122451121ADD12242A
:10028B00301203EE12044C122500122470D53923C0
:10029B00753906B20330030912072112068D0202CB
:1002AB00AF1201ADD53A0C753A041214C71201996D
:1002BB001201A3D0E0FBD0E0FAD0E0F9D0E0F8D007
:1002CB00E0F574D0E0F583D0E0F582D0E0F5F0D026
:1002DB00D0D0E0D2AF32E54FB4021130240ED2872A
:1002EB00C282054DD2A2121F4A02202F22E555755C
:1002FB00F001241084E5F0B40014E54FB40006754A
:10030B00568002037EB4020675568002037E22E5F8
:10031B005575F001241084E5F0B4000BE54FB400E3
:10032B000675565002037E22E55575F002241084A3
:10033B00E5F0B4000BE54FB4000675562202037EC0
:10034B0022E55575F004241084E5F0B4000BE54F5D
:10035B00B4000675561002037E22E55575F008248D
:10036B001084E5F0B4000BE54FB400067556070298
:0E037B00037E22200C0C302409D2B6C280D2A0
:10038900041211D0D21B85525022E55A75F01E84F1
:10039900B40403020365B4050302034CB406030263
:1003A9000333B4070302031AB4080302031A22E54C
:1003B90059B40F030203C2500574010203D0C39458
:1003C9000F8556F0842401F55222E559B40F030232
:1003D90003DD500574010203EBC3940F8556F084C5
:1003E9002401F55322D53C0302041BD53C03020426
:1003F9001BD53C0302041BD53C0302041BD53C035B
:1004090002041BD53C0302041BD53C0302041BD583
:100419003C0DD53D0A85483C85493D054FD2013003
:1004290001201202E1301B0FD5500CC21B202007FE
:10043900302404C2B6D280121D511203931203B89C
:10044900C20122D53E0302046DD53E0302046DD5D7
:100459003E0302046DD53E0302046DD53E0302043A
:100469006DD53E0DD53F0A85483E85493F054ED29B
:100479000030000B1204891205811203D3C2002235
:10048900201A0122D5500CC21A202007302404C298
:10049900B6D28022E55575F002241084E5F0B40047
:1004A90014E54EB4000675568002056CB402147545
:1004B900568002056CB4010BE54EB40106755680F1
:1004C90002056C22E55575F004241084E5F0B401A9
:1004D9000BE54EB4002275567802056CB4020BE5A3
:1004E9004EB4011475567802056CB4030BE54EB48D
:1004F900020675567802056C22E55575F008241038
:1005090084E5F0B4010BE54EB400227556300205BE
:100519006CB4030BE54EB4021475563002056CB485
:10052900060BE54EB4010675563002056C22E555F9
:1005390075F010241084E5F0B4010BE54EB40022E7
:1005490075561502056CB4060BE54EB401147556C3
:100559001502056CB40B0BE54EB40206755615026F
:10056900056C22200C0C302409D2B6C280D20412A8
:1005790011D0D21A85535022E55A75F01E84B40061
:10058900030204CDB401030204CDB402030205023F
:10059900B40303020537227563F71202367563DF68
:1005A9001202367563FF7564F71202367564FD121F
:1005B90002367564FF7565DF1202367565FD120234
:1005C9003675657F1202367565FF75637F120236CF
:1005D9007563FD1202367563FF7564DF12023675A5
:1005E900647F1202367564FF7565F7120236756508
:1005F900FF227563F31202367563CF1202367563F3
:10060900FF7564F31202367564FC1202367564FFD5
:100619007565CF1202367565FC12023675653F1293
:1006290002367565FF75633F1202367563FC120267
:10063900367563FF7564CF12023675643F12023650
:100649007564FF7565F31202367565FF22756300DF
:100659001201AD7563001201AD7563001201AD752C
:0D06690063551201AD7563001201AD75639C
:10067600001201AD7563001201AD7565551201AD2D
:100686007564001201AD22E546B400050546020672
:10069600A5B4010505460206C475460002070274A4
:1006A600FE7908339283D285C285D9F7C2B7D2B70D
:1006B6007908A2A133D2A6C2A6D9F7F5692274FD9C
:1006C6007908339283D285C285D9F7C2B7D2B77972
:1006D60008A2A133D2A6C2A6D9F7F56A2274FB797D
:1006E60008339283D285C285D9F7C2B7D2B77908C3
:1006F600A2A133D2A6C2A6D9F7F56B2274F7790860
:10070600339283D285C285D9F7C2B7D2B77908A208
:10071600A133D2A6C2A6D9F7F56C22E547B40005E7
:100726000547020751B40105054702076FB40205E4
:100736000547020791B4030505470207B3B404054C
:1007460005470207DD7547000207FBC2A3C286C242
:10075600B0D2A57914D9FEC2A57908C2A6D2A6A29E
:10076600A433D9F7C2A6F55D22D2A3C286C2B0D2FF
:10077600A57914D9FEC2A57908C2A6D2A6A2A43329
:10078600D9F7C2A630280122F55922C2A3D286C2C1
:10079600B0D2A57914D9FEC2A57908C2A6D2A6A25E
:1007A600A433D9F7C2A630280122F55A22D2A3C211
:1007B60086D2B0D2A57914D9FEC2A57908C2A6D22E
:1007C600A6A2A433D9F7C2A63028030207D6F55B42
:1007D60030290122F55C22D2A3D286C2B0D2A579F5
:1007E60014D9FEC2A57908C2A6D2A6A2A433D9F707
:1007F600C2A6F55E22C2A3C286D2B0D2A57914D90A
:10080600FEC2A57908C2A6D2A6A2A433D9F7C2A66B
:10081600F55F2212084312085112083512085F12BA
:10082600086D12087B12088912089A1208AB22E595
:100836006B30E4012220E60122756D0022E56B2073
:10084600E4012220E60122756D0122E56B20E40118
:100856002230E60122756D0222E56A30E30122208C
:10086600E50122756E0022E56A20E3012220E501FA
:1008760022756E0122E56A20E3012230E501227528
:100886006E0222E56C30E6012220E5012274019019
:10089600002FF022E56C20E6012220E501227402F9
:1008A60090002FF022E56C20E6012230E50122744B
:1008B6000490002FF022E56E7017C22EC22DD20FC3
:1008C6001208D8120A1112093D120B071209E4D2B6
:1008D6002C22302907900031E00208E4E55CB47868
:1008E600030208EF50030208F1747975F01784B417
:1008F600000C756600C2B1C2B3C2B5C2B422B4015F
:100906000C756601D2B1C2B3C2B5C2B422B4020C30
:10091600756602C2B1D2B3C2B5C2B422B4030C75B5
:100926006603C2B1C2B3D2B5C2B422756604C2B1FF
:10093600C2B3C2B5D2B422E56675F030A42567F518
:100946006022E56AF430E009757001D22A1209EDD9
:100956002230E109757000D22A1209ED2230E2092F
:10096600757002D22A1209ED2230E609757003D29B
:100976002A1209ED22E569F430E009757006D22ADB
:100986001209ED2230E109757009D22A1209ED2209
:1009960030E20975700AD22A1209ED2230E3097590
:1009A6007007D22A1209ED2230E40975700BD22A9B
:1009B6001209ED2230E509757008D22A1209ED22D6
:1009C60030E609757005D22A1209ED2230E709755D
:1009D6007004D22A1209ED22C22A1209ED22202A17
:0E09E60003D2A022C2A022E570202A05C2E79B
:1009F400F56822D2E7F56822900032E020E707C2CA
:100A04002AC2E7F57022D22AC2E7F57022302906FD
:100A14001209FC020A20120948020A20E570B401F6
:100A24001075670412093D75637F7564FF7565FF72
:100A340022B4001075670012093D7563F77564FFF1
:100A44007565FF22B4021075670812093D7563DFEE
:100A54007564FF7565FF22B4031075670C12093DB8
:100A64007563FD7564FF7565FF22B406107567181C
:100A740012093D7563FF7564DF7565FF22B40910C3
:100A840075672412093D7563FF7564FF7565FD2262
:100A9400B40A1075672812093D7563FF7564FF7504
:100AA40065F722B4071075671C12093D7563FF755D
:100AB40064FF7565DF22B40B1075672C12093D7550
:100AC40063FF7564FF75657F22B408107567201293
:100AD400093D7563FF75647F7565FF22B405107564
:100AE400671412093D7563FF7564FD7565FF22B4D3
:100AF400041075671012093D7563FF7564F7756519
:100B0400FF2222E570120CE722E56E7003D20F2259
:100B1400E56DB40212D22CC22EC22D300F05120E76
:100B2400B2C20F120CCA22D20F22E55EB4380302FD
:100B34000B385003790022B43C03020B4350037971
:100B44000122B44103020B4E5003790222B445033F
:100B5400020B595003790322B44A03020B64500375
:100B6400790422B44E03020B6F5003790522B45367
:100B740003020B7A5003790622B45703020B855003
:100B840003790722B45C03020B905003790822B462
:100B94006003020B9B5003790922B46503020BA680
:100BA4005003790A22B46A03020BB15003790B2271
:100BB400790B22120B2EE9900033F0120CC5120EA1
:100BC400B222900033E0F574120B2EE9B5740302DF
:100BD4000BF0E55EB43404120BB7225003020BF0A1
:100BE400B46B03020BF05004120BB722E56AF43025
:100BF400E00E200E51D20E7901120CC5120EB22253
:100C040030E10E200E40D20E7900120CC5120EB245
:100C14002230E20E200E2FD20E7902120CC5120ED3
:100C2400B22230E60E200E1ED20E7903120CC5122B
:100C34000EB222E569F430E00E200E0AD20E7906D7
:100C4400120CC5120EB22230E10E200E70D20E79B3
:100C540009120CC5120EB22230E20E200E5FD20E23
:100C6400790A120CC5120EB22230E30E200E4ED2B7
:100C74000E7907120CC5120EB22230E40E200E3D7E
:100C8400D20E790B120CC5120EB22230E50E200ED4
:100C94002CD20E7908120CC5120EB22230E60E20A8
:100CA4000E1BD20E7905120CC5120EB22230E70EBD
:100CB400200E0AD20E7904120CC5120EB222C20EF4
:100CC400228968897022302911900032E0C2E7B588
:100CD400700122D20FF570020EB2020BC6E570123B
:100CE4000CE722B4010A75637F7564FF7565FF2202
:100CF400B4000A7563F77564FF7565FF22B4020AD0
:100D04007563DF7564FF7565FF22B4030A7563FDBF
:100D14007564FF7565FF22B4060A7563FF7564DFA9
:100D24007565FF22B4090A7563FF7564FF7565FD77
:100D340022B40A0A7563FF7564FF7565F722B40768
:100D44000A7563FF7564FF7565DF22B40B0A75636A
:100D5400FF7564FF75657F22B4080A7563FF7564C7
:100D64007F7565FF22B4050A7563FF7564FD7565BB
:100D7400FF22B4040A7563FF7564F77565FF2222C8
:100D8400B4010A75633F7564FF7565FF22B4000AF8
:100D94007563F37564FF7565FF22B4020A7563CF4A
:100DA4007564FF7565FF22B4030A7563FC7564FFFF
:100DB4007565FF22B4060A7563FF7564CF7565FF18
:100DC40022B4090A7563FF7564FF7565FC22B40AD1
:100DD4000A7563FF7564FF7565F322B4070A7563CA
:100DE400FF7564FF7565CF22B40B0A7563FF7564E4
:100DF400FF75653F22B4080A7563FF75643F756526
:100E0400FF22B4050A7563FF7564FC7565FF22B49F
:100E1400040A7563FF7564F37565FF2222B4010942
:100E2400E563C2E7D2E6F56322B40009E563C2E3F1
:100E3400D2E2F56322B40209E563C2E5D2E4F563C4
:100E440022B40309E563C2E1D2E0F56322B40609E2
:100E5400E564C2E5D2E4F56422B40909E565C2E1BA
:100E6400D2E0F56522B40A09E565C2E3D2E2F5658C
:100E740022B40709E565C2E5D2E4F56522B40B099D
:100E8400E565C2E7D2E6F56522B40809E564C2E780
:100E9400D2E6F56422B40509E564C2E1D2E0F56462
:100EA40022B40409E564C2E3D2E2F5642222120EFC
:100EB400BE1210FDE570120E2122790C900022055D
:100EC400A2900016E0A320E70605A2F0A305A2D98C
:100ED400F305A27480F022E56E700122E56DB40181
:100EE40016D22CC22F1216F61216D9202E09120E63
:100EF400FC120FC6120EBE22E56AF430E00D200D7E
:100F04004CD20D900017E0B2E7F02230E10D200D35
:100F14003CD20D900016E0B2E7F02230E20D200D35
:100F24002CD20D900018E0B2E7F02230E60D200D2F
:100F34001CD20D900019E0B2E7F022E569F430E02C
:100F44000D200D09D20D90001CE0B2E7F02230E133
:100F54000D200D6DD20D90001FE0B2E7F02230E2BB
:100F64000D200D5DD20D900020E0B2E7F02230E3B9
:100F74000D200D4DD20D90001DE0B2E7F02230E4BB
:100F84000D200D3DD20D900021E0B2E7F02230E5B6
:100F94000D200D2DD20D90001EE0B2E7F02230E6B8
:100FA4000D200D1DD20D90001BE0B2E7F02230E7BA
:100FB4000D200D0DD20D90001AE0B2E7F022C20D03
:100FC4002222900017E020E70BE563C2E7C2E6F5B2
:100FD40063020FE0E563D2E7D2E6F563900016E022
:100FE40020E70BE563C2E3C2E2F563020FFAE563AF
:100FF400D2E3D2E2F563900018E020E70BE563C288
:10100400E5C2E4F563021014E563D2E5D2E4F563C6
:10101400900019E020E70BE563C2E1C2E0F563024A
:10102400102EE563D2E1D2E0F56390001CE020E7E6
:101034000BE564C2E5C2E4F564021048E564D2E558
:10104400D2E4F56490001FE020E70BE565C2E1C23D
:10105400E0F565021062E565D2E1D2E0F565900045
:0710640020E020E70BE56529
:10106B00C2E3C2E2F56502107CE565D2E3D2E2F59C
:10107B006590001DE020E70BE565C2E5C2E4F56570
:10108B00021096E565D2E5D2E4F565900021E020EB
:10109B00E70BE565C2E7C2E6F5650210B0E565D280
:1010AB00E7D2E6F56590001EE020E70BE564C2E7AA
:1010BB00C2E6F5640210CAE564D2E7D2E6F56490A5
:1010CB00001BE020E70BE564C2E1C2E0F56402100F
:1010DB00E4E564D2E1D2E0F56490001AE020E70980
:1010EB00E564C2E3C2E2F56422E564D2E3D2E2F541
:1010FB0064227563FF7564FF7565FF900022E0FA4B
:10110B00E0F92570C39AB40C0302111C50030211B1
:10111B001FC3940C121128A3E930E7E422B4010990
:10112B00E563C2E7C2E6F56322B40009E563C2E3F7
:10113B00C2E2F56322B40209E563C2E5C2E4F563DA
:10114B0022B40309E563C2E1C2E0F56322B40609E8
:10115B00E564C2E5C2E4F56422B40909E565C2E1C0
:10116B00C2E0F56522B40A09E565C2E3C2E2F565A2
:10117B0022B40709E565C2E5C2E4F56522B40B09A3
:10118B00E565C2E7C2E6F56522B40809E564C2E786
:10119B00C2E6F56422B40509E564C2E1C2E0F56478
:1011AB0022B40408E564C2E3C2E2F56422E56EB43E
:1011BB000109E56B30E5012212152522E56EB4021B
:1011CB00031215252230040DC204202008E56EB44D
:1011DB00020312152522E55DB402030211EB500345
:1011EB00790022B406030211F65003790122B40AE6
:1011FB00030212015003790222B40F0302120C50A6
:10120B0003790322B413030212175003790422B497
:10121B0018030212225003790522B41D0302122D6A
:10122B005003790622B421030212385003790722A6
:10123B00B425030212435003790822B42A03021285
:10124B004E5003790922B42E030212595003790A26
:10125B0022B433030212645003790B22790B22E57B
:10126B005DB437030212745003790022B43C0302BD
:10127B00127F5003790122B4400302128A50037982
:10128B000222B445030212955003790322B4490399
:10129B000212A05003790422B44E030212AB500386
:1012AB00790522B452030212B65003790622B457C1
:1012BB00030212C15003790722B45B030212CC5014
:1012CB0003790822B460030212D75003790922B4C0
:1012DB0064030212E25003790A22B468030212ED8E
:1012EB005003790B22790B22E55DB46D030212FDDD
:1012FB005003790022B471030213085003790122C1
:10130B00B476030213135003790222B47A03021347
:10131B001E5003790322B47E030213295003790470
:10132B0022B483030213345003790522B4870302DA
:10133B00133F5003790622B48C0302134A500379EE
:10134B000722B490030213555003790822B4950376
:10135B000213605003790922B4990302136B5003F3
:10136B00790A22B49E030213765003790B22790B70
:10137B0022E55DB4A2030213865003790022B4A7C1
:10138B00030213915003790122B4AB0302139C5057
:10139B0003790222B4B0030213A75003790322B4DA
:1013AB00B4030213B25003790422B4B9030213BD80
:1013BB005003790522B4BD030213C85003790622EA
:1013CB00B4C1030213D35003790722B4C60302132B
:0E13DB00DE5003790822B4CA030213E950035E
:1013E900790922B4CF030213F45003790A22B4D441
:1013F900030213FF5003790B22790B22E55DB4D860
:101409000302140F5003790022B4DC0302141A50AA
:1014190003790122B4E1030214255003790222B4AD
:10142900E5030214305003790322B4EA0302143BA2
:101439005003790422B4EE030214465003790522BD
:10144900B4F3030214515003790622B4F7030214CA
:101459005C5003790722B4FC03021467500379082E
:1014690022B4FE030214725003790922790A22E593
:101479005DB4330302148250091211E189747400B6
:10148900FB22B46803021493500912126A89747416
:1014990001FB22B49E030214A450091212F38974A9
:1014A9007402FB22B4D4030214B5500912137C89C7
:1014B900747403FB2212140589747404FB22121438
:1014C900787A00900022E020E70DB574030214E158
:1014D9005006A3FA0214CFEA2570F9BB0424B40A12
:1014E9000302150B401C7A00900022E020E70D252D
:1014F90070B40A06E0FAA30214F440F8EA2570026F
:10150900150CE975F004A4F9EB75F030A4FAE92A91
:10151900900036F022F560EB1208F522900036E0D3
:10152900F560EB1208F522E56E700122E56DB40055
:101539000DC22EC22D1219E212164312157A22E596
:101549006E700122E56DB401151219E230300F12E7
:1015590016BD120EFC120FC6120EBEC23022B40204
:101569000F1219E23031091216BD120EB2C2312220
:1015790022202C0122E572120D84E573120E21C27C
:101589002CE56E700122E56DB40006302F031216AA
:10159900BD22E56AF430E114E571C2E0C2E1C2E2BC
:1015A900C2E3F571757200D22CD22F2230E214E514
:1015B90071D2E0C2E1C2E2C2E3F571757202D22CC6
:1015C900D22F22E569F430E114E571D2E0C2E1D20B
:1015D900E2C2E3F571757209D22CD22F2230E314DD
:1015E900E571C2E0C2E1D2E2C2E3F571757207D2D8
:1015F9002CD22F2230E414E571C2E0D2E1D2E2C24A
:10160900E3F57175720BD22CD22F2230E614E571F5
:10161900D2E0D2E1C2E2C2E3F571757205D22CD2F1
:101629002F2230E714E571C2E0D2E1C2E2C2E3F54C
:1016390071757204D22CD22F2222E56AF430E0149B
:10164900E571C2E4C2E5C2E6C2E7F571757301D27C
:101659002CD22F2230E614E571D2E4C2E5C2E6C2EB
:10166900E7F571757303D22CD22F22E569F430E0C6
:1016790014E571C2E4D2E5C2E6C2E7F571757306F5
:10168900D22CD22F2230E514E571D2E4D2E5C2E69C
:10169900C2E7F571757308D22CD22F2230E214E516
:1016A90071C2E4C2E5D2E6C2E7F57175730AD22CBC
:1016B900D22F2222E571C2E0C2E1C2E2C2E3C4B480
:1016C9000407122122120EBE2212214D120EBE2231
:1016D900E56B30E303C22B22202B11D22B202D05E1
:1016E900D22ED22D22C22E1220F2C22D22202E015C
:1016F90022E571C2E4C2E5D2E6C2E7F57175730A63
:1017090012159B12157A22900034E0F5741219E231
:10171900E9B5740302173AE55FB434041219E222F9
:10172900500302173AB4540302173A50041219E24B
:101739002212159B22E55FB437030217485007743C
:1017490001900035F022B43C030217575007740288
:0E175900900035F022B440030217665007746A
:1017670003900035F022B44503021775500774043F
:10177700900035F022B4490302178450077405908E
:101787000035F022B44E03021793500774069000F9
:1017970035F022B452030217A250077407900035A0
:1017A700F02222E55FB457030217B4500774019083
:1017B7000035F022B45B030217C350077402900090
:1017C70035F022B460030217D25007740390003536
:1017D700F022B464030217E150077404900035F057
:1017E70022B468030217F050077405900035F02201
:1017F700B46D030217FF50077406900035F022B44A
:10180700710302180E50077407900035F02222E585
:101817005FB4760302182050077401900035F02258
:10182700B47A0302182F50077402900035F022B4DF
:101837007E0302183E50077403900035F022B483EC
:101847000302184D50077404900035F022B4870343
:1018570002185C50077405900035F022B48C03021F
:10186700186B50077406900035F022B490030218E5
:101877007A50077407900035F02222E55FB495038C
:1018870002188C50077401900035F022B4990302B6
:10189700189B50077402900035F022B49E0302187B
:1018A700AA50077403900035F022B4A2030218B9B6
:1018B70050077404900035F022B4A7030218C850EB
:1018C700077405900035F022B4AB030218D7500710
:1018D7007406900035F022B4B0030218E65007747E
:1018E70007900035F02222E55FB4B4030218F850E0
:1018F700077401900035F022B4B9030219075007A5
:101907007402900035F022B4BD0302191650077413
:1019170003900035F022B4C103021925500774045F
:10192700900035F022B4C6030219345007740590AD
:101937000035F022B4CA0302194350077406900019
:1019470035F022B4CF0302195250077407900035BF
:10195700F02222E55FB4330122500122B452030280
:10196700196B501312173EE571C2E4C2E5C2E6C215
:10197700E7F57175730122B47103021986501312CA
:1019870017AAE571D2E4C2E5C2E6C2E7F57175733D
:101997000322B490030219A15013121816E571C25D
:1019A700E4D2E5C2E6C2E7F57175730622B4B00367
:1019B7000219BC5013121882E571D2E4D2E5C2E6CF
:1019C700C2E7F571757308221218EEE571C2E4C219
:1019D700E5D2E6C2E7F57175730A2212195A90002B
:1019E70034E0F575900035E0B5750EE56E700122AF
:1019F700E56DB4000312159B22D22F900035E090BD
:101A07000034F0B40103021A125016E571C2E0C2A5
:101A1700E1C2E2C2E3F571757200D22CD231D23045
:101A270022B40203021A305016E571D2E0C2E1C2B5
:101A3700E2C2E3F571757202D22CD231D23022B4F0
:101A47000303021A4E5016E571C2E0D2E1C2E2C2A8
:101A5700E3F571757204D22CD231D23022B404036B
:101A6700021A6C5016E571D2E0D2E1C2E2C2E3F588
:101A770071757205D22CD231D23022B40503021A05
:101A87008A5016E571C2E0C2E1D2E2C2E3F5717590
:101A97007207D22CD231D23022B40603021AA850D0
:101AA70016E571D2E0C2E1D2E2C2E3F571757209BF
:101AB700D22CD231D23022B40703021AC65016E50F
:101AC70071C2E0D2E1D2E2C2E3F57175720BD22C9A
:0E1AD700D231D230222230231A054C121C7656
:101AE500121B19121B52121AFD121B41121C241231
:101AF5001C8A121CEEC22322E54C75F01824608462
:101B0500E5F0B40C06202402C28222B4000520248C
:101B150002D28222E54C75F006246084E5F0B40318
:101B25000C202408D287121F4A02202F22B4000B52
:101B3500202408C287121F4A02202F22E54CB460D8
:101B45000B754C00202405C2A2121F232220240B52
:101B5500E54CB4000122B40302D2A222E54C75F093
:101B650030246084E5F0B400097557087562600299
:101B75001C6122E54C75F018246084E5F0B4000979
:101B850075570F756260021C6122E54C75F00C24D7
:101B95006084E5F0B4000975571E756260021C612A
:101BA50022E54C75F006246084E5F0B4000975570C
:101BB5003C756260021C6122E54C75F0032460846B
:101BC500E5F0B40009755778756260021C6122E57D
:101BD5004C75F020246084E5F0B4000675570A02C0
:101BE5001C6122E54C75F010246084E5F0B4000614
:101BF500755714021C6122E54C75F008246084E5D4
:101C0500F0B40006755728021C6122E54C75F004F6
:101C1500246084E5F0B40006755750021C6122E586
:101C25005A75F01E84B40003021C10B40103021B94
:101C3500FCB40203021BE8B40303021BD4B404037F
:101C4500021B61B40503021B78B40603021B8FB4A3
:101C55000703021BA6B40803021BBD22200C0C209F
:101C65002409D2B6C280D2041211D0D21C85545197
:101C750022201C0122D5510CC21C2020072024043F
:101C8500C2B6D28022E559B40F03021C94500574E4
:101C950001021CA2C3940F8557F0842401F554E575
:101CA50057B4800375540122E55975F00484B400D6
:101CB50005D20CC22022B43F05C20CD22022C20C90
:101CC500C22022E55BB4A003021CDC500A122347A4
:101CD50075F002A4021CEBB4C803021CEA500612FC
:101CE50023D2021CEB22F56122E55BB4C803021C7A
:101CF500F84032B4FA03021D00502BE54C75F00391
:101D0500246084E5F0B4001DE54C75F06024608422
:101D1500E5F0FAC374609A75F00284F5F07405A4D1
:101D2500202402F56122E54C75F003246084E5F07A
:101D3500B40018E54C75F060246084E5F075F00298
:101D450084F5F07405A4202402F56122E55BB4C88E
:101D550003021D5B4019B4FA03021D63501274207F
:101D6500C3954D75F008A412233E302402F5612277
:101D7500E54D75F008A412233E302402F5612220BA
:101D85002406E54CFB021DAFE54D75F003A4FB02EF
:101D95001DAF20240EE54C75F0038475F002A4FBFD
:101DA500021DAFE54D75F002A4FB858232858333B4
:101DB50075340075350078328B36753700793612F3
:101DC500225B868208868322E571C2E0C2E1C2E217
:101DD500C2E3C4B40004121DF522B40104121E2D81
:101DE50022B40204121E6522B40304121E9D22228F
:101DF500E571C2E4C2E5C2E6C2E7B40004902596E7
:101E050022B401049025A222B402049025AE22B486
:101E150003049025BA22B404049025C622B405040F
:101E25009025D2229025DE22E571C2E4C2E5C2E604
:101E3500C2E7B400049025EA22B401049025F622F5
:101E4500B4020490260222B4030490260E22B404A0
:0F1E55000490261A22B4050490262622902632E5
:101E640022E571C2E4C2E5C2E6C2E7B400049026EA
:101E74003E22B4010490264A22B40204902656223B
:101E8400B4030490266222B4040490266E22B4059E
:101E94000490267A2290268622E571C2E4C2E5C225
:101EA400E6C2E7B4000490269222B4010490269E70
:101EB40022B402049026AA22B403049026B622B4C3
:101EC40004049026C222B405049026CE229026DA79
:101ED40022E571C2E4C2E5C2E6C2E7B400049000A0
:101EE4000022B4010490000C22B4020490001822D1
:101EF400B4030490002422B4040490003022B405F6
:101F04000490003C2290004822E56C30E403C2288F
:101F140022D22822E56A30E403C22922D2292205EA
:101F24006F121F30121F3C900030F02290002FE0FF
:101F340004B56F03756F012290002FE0B56F012285
:101F4400400122F56F2220282290002FE0B40412D1
:101F5400121F81121D84E559F0A3E55AF0A3E55B35
:101F6400F022B40203021F9C021FEA121F81121DF9
:101F740084E0F559A3E0F55AA3E0F55B22E56FB4DC
:101F8400010490003722B4020490009A22B403049E
:101F94009000FD2290016022E56FB4012390003788
:101FA400121D84E559F0A3E55AF0A3E55BF0900017
:101FB400FD121D84E559F0A3E55AF0A3E55BF02278
:101FC400B4022290009A121D84E559F0A3E55AF058
:101FD400A3E55BF0900160121D84E559F0A3E55A76
:101FE400F0A3E55BF022900037121D84E559F0A3BD
:101FF400E55AF0A3E55BF090009A121D84E559F0D0
:10200400A3E55AF0A3E55BF09000FD121D84E559A9
:10201400F0A3E55AF0A3E55BF0900160121D84E59E
:1020240059F0A3E55AF0A3E55BF02220291E9000A5
:102034002FE0B4040E122064121D97E55CF0A3E5B2
:1020440068F022B4020302207F0220BD1220641231
:102054001D97E0F9A3E0900032F0E9900031F022FE
:10206400E56FB401049001C322B402049002052276
:10207400B403049002472290028922E56FB4011B45
:102084009001C3121D97E55CF0A3E568F090024748
:10209400121D97E55CF0A3E568F022B4021A9002E1
:1020A40005121D97E55CF0A3E568F0900289121D06
:1020B40097E55CF0A3E568F0229001C3121D97E553
:1020C4005CF0A3E568F0900205121D97E55CF0A3AF
:1020D400E568F0900247121D97E55CF0A3E568F00F
:1020E400900289121D97E55CF0A3E568F022C2AF67
:1020F400790C90001605A2121ED505A2122106D253
:10210400AF22E0A343D20205A2F0A375D25275D246
:10211400A2E5D220E0FB53D2FD05A2D9E522C2AF4D
:10212400790C121ED505A290001605A2122136D2F2
:10213400AF2243D202438E20E0A353D2FD538EDF5D
:1021440005A2F0A305A2D9EA22C2AF790C7B001242
:102154001DCD05A290001605A2122163D2AF22EB79
:102164009305A2F0A305A20BD9F522E56AF430E1A8
:1021740063E569F430E45D7405120CE7120236126B
:1021840002361202361202361202361202361202D7
:1021940036C2AF1221D91221EB1221FB12220B12EB
:1021A400221B12222B12223B12224BD2AF120236D6
:1021B4001202361202361202361202361202361297
:1021C4000236120236120236120236120236120297
:0E21D4003612023622790C7B0090258A05A275
:1021E20090001605A212216322790C90001605A216
:1021F20090000005A212210622790C90001605A279
:1022020090000C05A212210622790C90001605A25C
:1022120090001805A212210622790C90001605A240
:1022220090002405A212210622790C90001605A224
:1022320090003005A212210622790C90001605A208
:1022420090003C05A212210622790C90001605A2EC
:1022520090004805A212210622E627F5270809E682
:1022620037F528782722C3E697F5270809E697F578
:10227200287827228627872908098628872A122272
:10228200FB782C22862C08862D08862E08862F871E
:102292002909872A12229E7827792E227530007505
:1022A20031101222E01222B11222D4D531F422C30B
:1022B200E52E9529E52F952AE5309400500122E577
:1022C2002E9529F52EE52F952AF52FE5309400F568
:1022D2003022B3E52733F527E52833F52822C3E575
:1022E2002C33F52CE52D33F52DE52E33F52EE52F88
:1022F20033F52FE53033F53022E5278529F0A4F5B3
:102302002C85F02DE528852AF0A4F52E85F02FE501
:10231200288529F0A4252DF52DE52E35F0F52EE59D
:102322002F3400F52FE527852AF0A4252DF52DE57C
:102332002E35F0F52EE52F3400F52F22B4F00122D0
:10234200400274F022B47801224002747822B43040
:1023520001224002743022900010E004B410027492
:1023620000F0900000A98229F582E022900014E09A
:10237200FA900011E004B40F0274FFF090256A9302
:102382002A900014F0900013E004B410027400F0DC
:10239200F9900014E0FA900000E58229F582EAF053
:1023A20022900014E0FA900012E004B4110274FFCB
:1023B200F0902579932A900014F012238722122399
:1023C2005954016008122359541F246022747F2239
:1023D20012235975F00584122350243022122359F6
:1023E2005401600D12235975F005841223502430D4
:1023F2002212235975F00584122350246022E56BC2
:1024020020E210D22430320FC282D287C2B6D280EA
:10241200C23222C224D232223009120542E542B42B
:10242200FF0B0543E543B4FF04C208C2092205407D
:10243200E540B4FF190541E541B4FF127540FF754F
:1024420041FF753CFF753DFF85404885414922E5C6
:102452006B30E103C20A22200A13D20A300906C2F3
:102462000912254922754200754300D20922E56B03
:1024720030E003C20B22200B48D20B302404C28767
:10248200D282E555240275F00284E5F0B400188585
:10249200404885414975400075410085483C854961
:0C24A2003D85483E85493F754F00754E52
:1024AE0000054D05551224C4D200D2013024061267
:1024BE001F4A02202F22E555B4100E755500754D9A
:1024CE0000302405C2A2121F2322E56B30E703C29F
:1024DE000622200608D206D226D2B6C2A222E56A6B
:1024EE0030E703C20722200708D207D226D2B6C28F
:1024FE00A2222024012220260122754000754100CF
:10250E0085483C85493D85483E85493F7555007552
:10251E004F00754E00754D00756F01C22622302496
:10252E00012220260122754200754300854A44850A
:10253E004B45754C00756F01C2262285423285438C
:10254E003375340075350078327536187537007965
:10255E0036122286864A08E604F54B2203002C0C1E
:10256E0001057E2133E6FF0B4D68146405150D5AE7
:10257E004B1B26351E1A96114042C8D50001020388
:10258E000405060708090A0B008102830405860765
:10259E0088098A0B008182830485860788898A8B45
:1025AE00008182830485860788098A8B0081828355
:1025BE000485860788898A0B0081828304850687B5
:1025CE0088898A0B008182838405868788890A8B95
:1025DE00008182030485860788090A8B0081020325
:1025EE008405860708898A0B008102038405860705
:1025FE0008890A8B008182038485860788898A8BE5
:10260E00008182038485860788098A8B0081820374
:10261E008485860788890A8B0081820384850687D4
:10262E0088890A8B008182038405060788890A8BB4
:10263E00008102038405860788090A8B0001820344
:10264E008405860708890A8B0081028304850607A4
:10265E0088098A0B008102038405068708098A0B04
:10266E00008102830405860788090A8B0081028394
:10267E000485068708890A8B0081028384058607F4
:10268E0088890A8B000182830405860708890A8BD4
:10269E00008102038405060708898A0B0001820364
:1026AE008485860708898A8B000182830405860744
:1026BE0008898A0B008102830405860708890A8B24
:1026CE00008102030485060708098A0B00018203B4
:1026DE000485060788090A8B464C414D4520544116
:1026EE004D45204D414348494E45204555524F20BA
:1026FE005241434B2056455253494F4E202D2032C6
:10270E003031302056455253494F4E20312E303104
:0D271E0020286329627920616D7065726565
:00000001FF
